S123E0008693B710398600B710248600B71035CEB600DF98CEB7FFDF9ACE0000DFAC8E0011
S123E0205FBDE31CCE0041DF69B610208A03B7102086D09768CC3F0DDD6BBDE18D7F00A40D
S123E0407C00A47F00A6B6103C84202717CEB5F8861CA703A103260CA701A60184102704E8
S123E060860197A67F00A5BDE08C96A6270597A5BDE08C7F00A5BDE350810D271996A62779
S123E080F297A5BDE350810D270C20E7BDE33DCEE584BDE45C397F00A796A58101270496A8
S123E0A0A697A70F8E005F7F00A47C00A4BDE44C863EBDE3695FBDE488CE006B3A811827C4
S123E0C0E2817F27DE810826055A2DD720E8810D26075D2717A7002013A7005CC1232F08ED
S123E0E0CEE5CEBDE45C20BB812F26CA7F00C07F00967F00975FCE006BDFAEBDE2DBBDE27B
S123E100C6CE008E3ABDE182A700810D2736BDE2EB2731BDE2CD5CC1082F09CEE5CEBDE420
S123E1205C7EE0A3812F26177D00C026095AD7A8CEE85B7EE17DCEE5E6BDE45C7EE0A3BD0B
S123E140E1DC20BAD7A8CEE492DFB0DEB018CE008EE600C1FF2609CEE5C8BDE45C7EE0A382
S123E1603CCB033ADFB0385F5CA60118A10026DB081808D1A82DF1DEB00909EE00AD007EFC
S123E180E0A381612D06817A2E02802039CE009CC6086F00085A2EFA39505958414243535B
S123E1A00002040607080901010100000001A600363CBDE369862DBDE369E607A60ECE00E7
S123E1C0603A4D2703BDE434BDE4433832393CCEE199BDE1AE08815326F8383936373CBD2D
S123E1E0E18281302D2281392F0A81412D1A81462E168B09840FCE0096C604680169005A30
S123E2002EF9AA01A70120037C00C0383332397F00C07F00A87F00967F0097BDE2DBBDE2A1
S123E220C6BDE1DC7D00C026087C00A8BDE2CD20ED397F00A87F00967F0097BDE488811845
S123E2402704817F26037EE0A37F00C0BDE1DC7D00C026057C00A820E2397D00A8270596FE
S123E26097BDE265398C103F27109C9825129C9A220E37E600C1FF332703BDE29BBDE28F41
S123E280A700A10027083CCEE5E1BDE45C383937C602F7103BA700C603201837C616F710C2
S123E2A03BC6FFE700C617200A37C606F7103BA700C60726015FF7103B333CCE0D0609266C
S123E2C0FD387F103B393CDEAEA60038393CDEAE0820043CDEAE09DFAE3839BDE2C6BDE25C
S123E2E0EB2605BDE2CD20F3810D39812C270681202702810939BDE2EB2702810D39BDE33D
S123E30050271881172605BDE35027FB817F270881182704810126037EE0A339CE00C41813
S123E320CEE336CC7E03A1002705A7001AEF013A8C010026F139865006CF7EE336363C96C6
S123E340A581002605BDE37F2003BDE3BE3832393C8655B7103A86AAB7103A96A52605BDB9
S123E360E38F2003BDE3D4383936373CD6A52605BDE39C2003BDE3EE3833327C00A9398662
S123E38030B7102B8600B7102C860CB7102D39B6102E84202705B6102F847F397D00A427E2
S123E3A0108D0E810D2604860A2006810A260E860DF6102EC58027F9847FB7102F393CCE19
S123E3C0B5F88600A701861CA703860BA702A600A6013839CEB5F8A6013684063227068653
S123E3E00197C2200484082704A600847F398D187D00A42712810D2606860A8D0B20088178
S123E4000A2604860D8D0139CEB5F8E601C5102604C54027F3847FA70039FFFFFFFFFFFF0D
S123E420FFFF44444444840F8B3081392F028B07BDE3693936A600368DE8328DE93208391B
S123E440BDE434BDE4348620BDE36939860DBDE3698600BDE369860D7F00A939BDE44C36E4
S123E460A60081042714BDE36908BDE35027F1811726EDBDE35027FB20E6323936BDE446CE
S123E48096A981142FF73239BDE3504D27FABDE3693905415353454DEA6805425245414B39
S123E4A0E6320442554C4BE6ED0742554C4B414C4CE6F10443414C4CF9410444554D50E6DC
S123E4C0FA0545454D4F44E78F0446494C4CE7DF02474FF99A0448454C50F54804484F53E5
S123E4E054FB15044C4F4144FBAD064D454D4F5259E847044D4F5645E91B064F4646534522
S123E50054FCB80750524F43454544F988085245474953544552FCF90653544F504154FA28
S123E52070055452414345FA2B06564552494659FBA5013FF5480558424F4F54FD69017E60
S123E540FDE10341534DEA68024246E7DF04434F5059E91B054552415345E6ED024D44E64F
S123E560FA024D4DE847025244FCF902524DFCF90452454144E91B02544DFB1504544553E8
S123E58054FDE2FF42554646414C4F20332E344158202D20434D442D313141205573657228
S123E5A0204661737420467269656E646C792041696420746F204C6F676963616C204F7061
S123E5C065726174696F6E04576861743F04546F6F204C6F6E670446756C6C044F702D20E1
S123E5E004726F6D2D04436F6D6D616E643F0442616420617267756D656E74044E6F2068BF
S123E6006F737420706F727404646F6E650463686B73756D206572726F72046572726F720A
S123E6202061646472200472637672206572726F7204BDE2DB2604BDE6C939812D2631BDE1
S123E640E2CDBDE2C6BDE2F62606BDE18D7EE632BDE20FBDE2F62707CEE5EFBDE45C39BD1A
S123E660E6D85D2B08CE009C3A6F006F017EE632BDE20FBDE2F62707CEE5EFBDE45C39BD29
S123E680E6D85D2CADDE96A60036863FBDE265E60032BDE265C13F270CDFB0CE00B0BDE46C
S123E6A040BDE6C9397F00967F00973CBDE6D8385D2A0ACEE5D7BDE45CBDE6C93918CE00B4
S123E6C09C183ACDEF007EE632BDE44CCE009CC604BDE4405A2EFA395FCE009C3AEE009CAC
S123E6E0962601395C5CC1062FEFC6FF39DE982003CE103F86FFBDE2A939DEAADFB0C6806C
S123E7003ADFB2BDE2DB2735BDE20F7D00A82726BDE2F62621DE96DFB0C6803ADFB2BDE2A5
S123E720DB271ABDE20F7D00A8270BBDE2DB2606DE96DFB22007CEE5EFBDE45C39DCB0DDA1
S123E740AAC4F0DDB0BDE44CCE00B0BDE440DEB05FBDE4435CC1102DF85FDEB03AA600810D
S123E760202504817A23028620BDE3695CC1102DE9BDE2FEDCB0C30010DDB01A93B2220E22
S123E7801A83000026BFDCB21A83FFF025B739BDE2DB2734BDE20F7D00A8273CBDE2F626FE
S123E7A037DC96DDB0C307FFDDB2BDE2DB2711BDE20F7D00A82721BDE2DB261CDE96DFB239
S123E7C0DEB0DF98DEB2DF9ABDE44CCE0098BDE440CE009ABDE44039CEE5EFBDE45C39BDDC
S123E7E0E2DBBDE20F7D00A8274FBDE2EB264ADE96DFB0BDE2DBBDE20F7D00A8273BBDE2C4
S123E800F62636DE96DFB286FF97C1BDE2DB2711BDE20F7D00A82721BDE2DB261C96979773
S123E820C1BDE2FEDEB096C1BDE265A10026119CB2270508DFB020E939CEE5EFBDE45C398A
S123E840CE00B0BDE44039BDE2DB2718BDE20FBDE2DB2707CEE5EFBDE45C397D00A82704E5
S123E860DE96DFAABDE44CCE00AABDE440DEAABDE4437F00967F0097BDE232BDE182DEAA41
S123E88081202731810A273E812B2743815E2748812D274481082740812F2745813D2741DC
S123E8A0814F2743810D276F812E276ECEE5E6BDE45C7EE864BDE25A08DFAA8FC40F27033C
S123E8C07EE86D7EE864BDE25A08DFAA7EE867BDE25A08DFAA7EE864BDE25A09DFAA7EE8FB
S123E8E064BDE25A7EE864DC9693AA81002606C1802313200881FF2604C1812409CEE5CE58
S123E900BDE45C7EE864830001D7C3BDE446CE00C3BDE4437EE864BDE25A39BDE20F7D008B
S123E920A8272BBDE2EB2626DE96DFB0BDE20F7D00A8271ABDE2F62615DE96DFB2BDE20F69
S123E940BDE2DB26097D00A8270BDE96200ACEE5EFBDE45C39DEB008DFB4DEB49CB02328EB
S123E9609CB22224DCB293B0D3B4DDB4DEB2BDE2FEA6003CDEB4BDE265A100262809DFB4E6
S123E980389CB0271F0920E6DEB0BDE2FEA6003CDEB4BDE265A100260C08DFB4389CB227DC
S123E9A0030820E63938CE00B4BDE44039E9BFE9D2E9E5E9F4EA01EA14EA2CEA47EA544970
S123E9C06D6D6564206D6F646520696C6C6567616C044572726F7220696E204D6E652074F8
S123E9E061626C6504496C6C6567616C20626974206F700442616420617267756D656E74D5
S123EA00044D6E656D6F6E6963206E6F7420666F756E6404556E6B6E6F776E20616464725C
S123EA20657373696E67206D6F646504496E64657865642061646472657373696E672061FA
S123EA407373756D65640453796E746178206572726F72044272616E6368206F7574206FF3
S123EA60662072616E676504CE0000DFBEBDE2DB2713BDE20FBDE2DB2707CEE9F4BDE45CDE
S123EA8039DE96DFBEDEBEDFB0BDE44CCE00B0BDE440BDF2BABDE47C863EBDE430BDEB49A5
S123EAA097BC815E2715812B2711812D270D812F2709813D27058100260439BDE44CBDE4E2
S123EAC046BDE446BDE446BDE446BDE446BDEB92C1052F08CEEA01BDE45C202FC100272EFE
S123EAE0BDEBD996B581FF2608CEEA01BDE45C201ABDEC1181002607CE0000DFB6200F4A64
S123EB0016CEE9AD3A3AEE00BDE45C7F00BC96BC815E2704812D2607DEBE09DFBE2027819C
S123EB200A2708812B2704810D261BDEB62606DEB0DFBE2011810A2704812B2605DEBE08A5
S123EB40DFB6DEB6DFBE7EEA855F860DCE006B3AA7005CC1232DF55FBDE488817F2731812F
S123EB6018272D81012729812E2725810327218104271D810826055A2EDE20CDCE006B3A49
S123EB80BDE182A700C1232C015CBDEBBE26C9394F3986209791CE006BDFAEBDE2DB5FBDFD
S123EBA0E2C6BDE2CDBDE2EB2713BDEBBE270EBDE182CE008E3AA7005CC1052FE239810A8A
S123EBC02716810D2712815E270E812F270A812B2706812D2702813D39CEEF3B18CE008E25
S123EBE02003C6063AA6008104260586FF97B53918A10026EDA60118A10126E6A60218A1EE
S123EC000226DFA60318A10326D8EC0497B4D7B539860497C17F00C2DEAE8C008E271BEC8F
S123EC200008812C26F4C1592606860297C1200AC1582606860197C12000BDE2DB81232629
S123EC4007BDE2CD860097C1D6B5C10226037EECAFC10126037EECB4C10526037EECBBC1F1
S123EC600826037EECEAC10726037EECF4C10326037EECFDC10426037EED0BC11526037E87
S123EC80ED3DC11026037EED5EC10926037EED67C11226037EED7FC11126037EED88C11316
S123ECA026037EEDA7C11426037EEDA78602398618BDEF3096B4BDEF304F39BDEF128104D9
S123ECC0260139DC96DEB00808DFB893B8DDB81A83007F23091A83FF80240386093996B4AC
S123ECE0BDEF3096B9BDEF304F3996C181002604860397C196C181002603860139860097C0
S123ED00C397B2861897B3BDEE433996C1810226098618BDEF30860197C196C1810126046F
S123ED20BDEEE33996B48B10BDEF30BDEF128104270ADC96BDEF3017BDEF304F3996C18132
S123ED40002604860397C196C1810226037C00C2861A97C397B286CD97B3BDEE433996C105
S123ED608100260386013996C181002604860397C1860097C397B286CD97B3BDEE433996BF
S123ED80C18100260386013996C1810226037C00C281002604860397C1861897C397B386AF
S123EDA01A97B2BDEE4339BDEE1D8100260386033996C1810226098618BDEF30860197C12F
S123EDC096B4BDEF30BDEF1281042601399697BDEF3096C181012606BDE2CDBDE2CDBDEFD4
S123EDE01281042601399697BDEF3096B5811426024F39BDEF128104260139DEB008DFB8AF
S123EE00DC9693B81A83007F230D1A83FF8024074FBDEF3086093917BDEF304F3996C1D603
S123EE20B581012601398102260139C114260796B4800897B439C113260796B4800C97B4DA
S123EE40394F3996C1810327138100272C810227418101274C8104275786063996C3BDEF57
S123EE602896B4BDEF30BDEF128104260139DC96BDEF3017BDEF304F3996C3BDEF2896B45D
S123EE80BDEF30BDEF1281042601399697BDEF304F3996B3BDEF2896B48B2097B4BDEEE373
S123EEA03996B2BDEF2896B48B2097B4BDEEE339BDEF12810426013996C3BDEF2896A88163
S123EEC0022E0E96B48B10BDEF309697BDEF304F3996B48B30BDEF30DC96BDEF3017BDEFAC
S123EEE0304F3996B4BDEF30BDEF128104260139812C2703860839BDE2CDBDE2C68159271D
S123EF000A81582706FEEA2CBDE45C9697BDEF304F39BDE20FBDEBBE2705BDE2EB26067DC8
S123EF2000A827013986043981002703BDEF3039DEB0BDE265BDE443DFB039414241201B04
S123EF4001414258203A01414259203A0241444341890341444342C903414444418B0341FA
S123EF60444442CB0341444444C308414E44418403414E4442C40341534C20680441534C5A
S123EF8041480141534C42580141534C4405014153522067044153524147014153524257DF
S123EFA00142434320240542434C521D14424353202505424551202705424745202C054240
S123EFC04754202E0542484920220542485320240542495441850342495442C503424C459B
S123EFE0202F05424C4F202505424C53202305424C54202D05424D49202B05424E452026F2
S123F0000542504C202A054252412020054252434C1F1342524E202105425253451E134284
S123F0205345541C14425352208D05425643202805425653202905434241201101434C43EC
S123F040200C01434C49200E01434C52206F04434C52414F01434C52425F01434C56200A00
S123F06001434D50418103434D5042C103434F4D206304434F4D414301434F4D425301437E
S123F0805044208315435058208C09435059208C11444141201901444543206A04444543B1
S123F0A0414A01444543425A01444553203401444558200901444559200902454F5241885F
S123F0C003454F5242C803464449560301494449560201494E43206C04494E43414C0149BF
S123F0E04E43425C01494E53203101494E58200801494E592008024A4D50206E044A535206
S123F100208D074C44414186034C444142C6034C444420CC084C4453208E084C445820CE89
S123F120094C445920CE114C534C2068044C534C4148014C534C4258014C534C4405014CE7
S123F14053522064044C53524144014C53524254014C53524404014D554C203D014E45471F
S123F1602060044E45474140014E45474250014E4F502001014F5241418A034F524142CA91
S123F18003505348413601505348423701505348583C01505348593C0250554C41320150E9
S123F1A0554C42330150554C58380150554C593802524F4C206904524F4C414901524F4C4F
S123F1C0425901524F52206604524F52414601524F52425601525449203B0152545320396E
S123F1E00153424120100153424341820353424342C203534543200D01534549200F015319
S123F2004556200B0153544141870753544142C70753544420CD0753544F50CF0153545385
S123F220208F0753545820CF1053545920CF1253554241800353554242C0035355424483C7
S123F24008535749203F0154414220160154415020060154424120170154504120070154C5
S123F2604553540001545354206D04545354414D01545354425D015453582030015453599C
S123F280203002545853203501545953203502574149203E01584744588F01584744598F96
S123F2A0024252534512164252434C131642534554141742434C52151704DEB0A600C60002
S123F2C08118270A811A270581CD26045C5C5C08DFB6D7C3A60097B408DFB6815F230F81B5
S123F2E08D270B818F270781CF27037EF385D6C3C1022504BDF53F39D6B45FBDF46E5D2663
S123F30004BDF53F3996B4818D2604C605200A818F270481CF2605C601BDF46ED6B5C1015B
S123F3202618D6C3C100270E96B4C602BDF46E5D2604BDF53F39BDF49139D6B5C105261018
S123F3407D00C32704BDF53F39BDF491BDF4C739D6B5C1172704C11626117D00C32704BD5D
S123F360F53F39BDF491BDF51F2006BDF491BDF4ABBDE446BDF51FD6B5C1132704C1162606
S123F38003BDF4C739817F222AD6C3C1022504BDF53F39846F5FBDF46E5D2604BDF53F3998
S123F3A0BDF49196B484F081602604BDF4AB39BDF52C398187270481C72604BDF53F39843F
S123F3C0CF5FBDF46E5D2604BDF53F3996B484CF818D2604C6072016818F2604C607200E1E
S123F3E081CF2604C61020068183260CC608BDF46E5D2604BDF53F39D6B5C1032708C10779
S123F4002704C108263196B484CF8183260FD6C3C1022509C615BDF46EC608D7B5D6C3C18F
S123F420012704C103260C96B484B081A02704BDF53F39BDF4E939D6C3C1012704C1022670
S123F4401396B484CFD6B5C1092604C6112002C612BDF46ED6C3C102250C96B484B081A05D
S123F4602704BDF53F39C608D7B5BDF4E939CEEF3BA104260F5D2704E1052608E605D7B521
S123F480DFBA5C3937C6063AE600C1043326E25F39DEBAA600BDE430A601BDE430A602BD93
S123F4A0E430A603BDE430BDE44639BDF51F862CBDE430D6C3C1012704C1032604865920D3
S123F4C0028658BDE43039DEB6E60008DFB65D2B033A2004095C26FCDFB8BDE4468624BDD2
S123F4E0E430CE00B8BDE44039BDF49196B484B0818026178623BDE430BDF51FD6B5C108B7
S123F500270139DEB6BDE434DFB63981902604BDF51F3981A02604BDF4AB39BDF52C39868D
S123F52024BDE430DEB6BDE434DFB6398624BDE430DEB6BDE440DFB639494C4C4F50043C1D
S123F540CEF539BDE45F3839CEF54FBDE45C3941534D205B3C616464723E5D20204C696EC1
S123F560652061736D2F64697361736D0D20205B2F2C3D5D202053616D6520616464722CC7
S123F580202020202020205B5E2C2D5D20205072657620616464722C202020202020205B19
S123F5A02B2C43544C4A5D204E65787420616464720D20205B43525D20204E657874206FE4
S123F5C070636F64652C2020202020202020202020202020202020202020202020202020B0
S123F5E0202020205B43544C412C2E5D2020517569740D4246203C61646472313E203C61B6
S123F600646472323E205B3C646174613E5D2020426C6F636B2066696C6C206D656D6F721E
S123F620790D4252205B2D5D5B3C616464723E5D2053657420757020626B70742074616261
S123F6406C650D42554C4B2020457261736520454550524F4D2C2020202020202020202016
S123F6602020202020202042554C4B414C4C2020457261736520454550524F4D20616E6434
S123F68020434F4E4649470D43414C4C205B3C616464723E5D2043616C6C20737562726F93
S123F6A07574696E650D474F205B3C616464723E5D204578656375746520636F6465206162
S123F6C07420616464722C202020202020202050524F434545442020436F6E74696E756544
S123F6E020657865637574696F6E0D45454D4F44205B3C616464723E205B3C616464723E7B
S123F7005D5D204D6F6469667920454550524F4D2072616E67650D4C4F41442C2056455228
S123F720494659205B545D203C686F73742064776E6C6420636F6D6D616E643E20204C6F26
S123F7406164206F722076657269667920532D7265636F7264730D4D44205B3C61646472A8
S123F760313E205B3C61646472323E5D5D20204D656D6F72792064756D700D4D4D205B3CAD
S123F780616464723E5D206F72205B3C616464723E5D2F20204D656D6F7279204D6F6469B0
S123F7A066790D20205B2F2C3D5D202053616D6520616464722C20205B5E2C2D2C43544CBB
S123F7C0485D205072657620616464722C20205B2B2C43544C4A2C53504143455D204E65F5
S123F7E0787420616464720D20203C616464723E4F20436F6D70757465206F666673657409
S123F8002C202020202020202020202020202020202020205B43525D2020517569740D4DCE
S123F8204F5645203C73313E203C73323E205B3C643E5D2020426C6F636B206D6F76650D98
S123F8404F4646534554205B2D5D3C6172673E20204F666673657420666F7220646F776E3E
S123F8606C6F61640D524D205B502C592C582C412C422C432C535D2020526567697374652B
S123F88072206D6F646966790D53544F504154203C616464723E2020547261636520756EFB
S123F8A074696C20616464720D54205B3C6E3E5D20205472616365206E20696E737472759D
S123F8C06374696F6E730D544D20205472616E73706172656E74206D6F6465202843544C24
S123F8E041203D20657869742C2043544C42203D2073656E642062726B290D5B43544C57CA
S123F9005D2020576169742C202020202020202020205B43544C582C44454C5D2041626F1F
S123F92072742020202020202020205B43525D20526570656174206C61737420636D640DBA
S123F94004BDE2DB2713BDE20FBDE2DB2707CEE5EFBDE45C39DE96DF60DE6909CCF96DED9B
S123F9600009DF69BDF9DE7F00C17EFACD360797680F32DD66DF6418DF629F699EB2BDFAAE
S123F9800BBDE44CBDE1CE39BDFAADBDE2FE7F00C17C00C1BDF9DE7EFACDBDE2DB2713BDFE
S123F9A0E20FBDE2DB2707CEE5EFBDE45C39DE96DF607F00C17C00C1BDF9DE7EFACD309EFB
S123F9C0B2BDFAECBDFA0BDE6009DF607D00C12606DE690808DF69BDE44CBDE1CE395FCEBE
S123F9E0009C18CE00B63A183AEE00270AA60018A700863FBDE265CB02C1062FE2DEF5DF9B
S123FA00B4867E97F4CEF9BEDFF5395FCE009C18CE00B63A183AEE00270618A600BDE2653F
S123FA20CB02C1062FE6DEB4DFF5397F00C37C00C37F00A9BDE2DB2713BDE20FBDE2DB27CE
S123FA4007CEE5EFBDE45C39969797C3D6C337DE60DFB0BDF2BA33D7C3BDFAADBDE2FEBDAB
S123FA60E47CBDE1CE7A00C32705BDE44C20DD39BDE2DB2718BDE20FBDE2DB2707CEE5EF79
S123FA80BDE45C397D00A82704DE96DFAADC601A93AA250ADCAAC3000A1A93602208BDFADC
S123FAA0ADBDE2FE20E7BDE44CBDE1CE39867E97D3CEFAE9DFF2966884BF9768C657FE1004
S123FAC00E3AFF101EB6102084FEB71020BF00B2BE0069FE00603CFE00623CFE00643CFCF6
S123FAE000663637B60068363B309EB2A6009768EC019767D766EC03DD64EC05DD62EC0700
S123FB00DD60C6083ADF69B610208A03B710208608B7100B3996A62607CEE5FCBDE45C3913
S123FB207F00A4BDFB7FBDE3504D27108101271781022605BDFB4B2003BDFB97BDFB8B4D80
S123FB4027E4BDE36920DF7C00A43996A78101270DCE102D1C00008D1D1D0000200DCEB5A4
S123FB60F8860FA7028D0F860BA702860DBDFB97860ABDFB973918CE0B29180926FC39D60F
S123FB80A537D6A7D7A5BDE33D2016D6A537D6A7D7A5BDE350200AD6A537D6A7D7A5BDE369
S123FBA06933D7A5397F00C17C00C120037F00C17F00C2BDE2DB2735BDE18281542616BD0B
S123FBC0E2CDBDE2C6BDE2D3810D26097F00A496A597A720187F00A4BDFB7FBDE2C6BDE2AC
S123FBE0CD36BDFB97BDE36932810D26EE96A791A52703BDE2FEBDFB8B4D27F1815326ED09
S123FC00BDFB8B4D27FA8139274E813126DF7F00C3BDFC9BD697C002BDFC9BBDFC9B37DCC9
S123FC2096D3AC8F3309BDFC9B085A271B7D00C226BB7D00C126059697BDE265A10027E680
S123FC40860297C2DFB420DE7D00C226A096C34C279B860397C22095BDFC9BD697BDFC9B16
S123FC605A26FAC664BDE2BA5A26FABDE350CC7E0DDD6B7C00A4CEE60996C281022608CEC6
S123FC8000B4BDE440201381012605CEE627200781032603CEE60EBDE45C39373CBDFB8B8E
S123FCA04D27FABDE1DCBDFB8B4D27FABDE1DC96979BC397C33833397F00C3BDE2DB272899
S123FCC0812D26097C00C3BDE2CDBDE2DBBDE20F7D00A8271DBDE2DB2618DC967D00C32776
S123FCE005CC00009396DDACBDE44CCE00ACBDE44039CEE5EFBDE45C39CEE199BDE2DBBDA5
S123FD00E182810D271CA100270EE60008C15326F5CEE5EFBDE45C393CBDE2CDBDE2DB3886
S123FD2026EFBDE1CEBDE44CBDE1AE7F00967F0097BDE232BDE2F62707CEE5EFBDE45C396E
S123FD40363C7D00A82714E607A60ECE00603A4D27059696A700089697A7003832E600C18B
S123FD6053270508810D26BD39BDE2DB260BCEC0FFDFB818CEC0002036BDE20F7D00A82789
S123FD802718DE96BDE2DB260C18DFB8DCB8C300FFDDB8201ABDE20F7D00A8270BDE96DFD4
S123FDA0B8BDE2DB26022007CEE5EFBDE45C39C6FFBDFDC718A600A72F1F2E80FC189CB8D7
S123FDC02704180820EE39CE10008602A708A7096F2D8622A72B860CA72DE72F1F2E80FC6D
S123FDE0393986FFB710007F00A4BDFB7F867FBDFB97860DBDFB977C00A4CE0070DFAE18AE
S123FE00CEFE1D18A60081042707A70008180820F27F00C1BDFBD58E005F7EC0B3636174C0
S111FE2020657662746573742E6F75740D041C
S123FF7C7EE0A37EE18D7EE1CE7EE1DC7EE20F7EE2327EE25A7EE2C67EE2CD7EE2D37EE26B
S107FF9CDB7EE2FE24
S123FFA07EE1827EE2EB7EE2F67EE33D7EE3507EE3697EE4227EE4267EE4307EE4347EE40C
S116FFC0437EE4407EE44C7EE45C7EE45F7EE4887EE31CB1
S123FFD600C400C700CA00CD00D000D300D600D900DC00DF00E200E500E800EB00EE00F15F
S10DFFF600F400F700FA00FDE0003B
S9030000FC
